:020000040000FA
:06000000703002303A28C6
:08000800A000030EA100831209
:1000100005191128831601178312B2308100B1012E
:100020002C2883160113831203140B190310A80D37
:10003000A90DAA0DAB0DAC0DAC16FF302C02031DA3
:100040002C28FA302B02031D2C2832152A08AF0069
:100050002908AE002808AD008B100B11210E83007B
:06006000A00E200E0900B5
:04006600003400342E
:0C007400203084008001840A80300402E7
:10008000031C3C28592183160C30850587018312F7
:10009000850187010730990000309A0010308316DF
:1000A0008E008312603083168F0083120030831617
:1000B00091009F008312C830831681008312313073
:1000C0009000003083168C00831210308B00BA2110
:1000D00081018E018F010B118B100B108C018B177E
:1000E000802032198C203B21B40B7E280310851907
:1000F0000314BA0DF0303A020319E420BD21702830
:1001000064003310B10A311F8B28AC01AB01AA0186
:10011000A901A801B101080032110130B7008B1309
:100120002030370783169B001C141A088312A40082
:100130001030370783169B001C141A088312A30083
:10014000A6000230A6060030370783169B001C1459
:100150001A088312A200A7000130A7068B17331CD0
:10016000B72822090339A200A309A409A509240874
:100170002F02031DDE2823082E02031DCC2822088F
:100180002D02031DDE2801303702031DCC283E1846
:10019000CC283E143F14802126082E02031DDE28A1
:1001A00027082D02031DDE2801303702031DDD283C
:1001B0003E1CDD283E103F14A421DE28B70A023081
:1001C0003702031808008F280130B600B400B500CC
:1001D000B70085018701B213B0218020B40B01293B
:1001E000031085190314BA0DF0303A0203192929B6
:1001F000B51F8501B51F8701B50B01299630B500E4
:100200003621321DED283211331C0B292D090339FB
:10021000AD00AE09AF092F1CED282D0830020319DF
:10022000ED282D08B0002E1EED288B132030370747
:10023000BC002F08BB00442110303707BC002E083B
:10024000BB00442100303707BC002D08BB0044210F
:100250008B1785018701B721B70AB6010130B500B8
:1002600002303702031CED28BA21080001303702A2
:100270000319A72108003F1C08003F101030BC00E4
:100280003E08BB00442108008B133B0883161C1555
:100290009A0083123C0883169B0055309D00AA30BB
:1002A0009D009C1464009C1852291C1183128B170A
:1002B0000800831610309B001C141A088312BE001D
:1002C000831620309B001C141A088312DF0083164B
:1002D00070309B001C141A088312D6000E07D7003A
:1002E0005707D8005607DB005807DA005607D90031
:1002F0005807D5007030BC005708BB0044210800E7
:100300000130BE000430C200C5000530C400C60084
:10031000CA000730C100C300C700C800C9005F1988
:10032000C1175F19C2175F19C317DF19C4175F1A06
:10033000C5175F1AC6175F1AC7175F1AC8175F1B62
:10034000C917DF18CA170800850187010800380996
:1003500033398500B80039093F398700B9000800F2
:1003600011308500B80013308700B9000800B801CB
:10037000B90108003E188021080001303E0503192C
:1003800008005F19C5295C1805165F19C929DC1812
:1003900085165F19CD295C190514DF19D129DC19DF
:1003A00085145F1AD5295C1A87145F1AD929DC1ABB
:1003B00007155F1ADD295C1B07145F1AE129DC1B96
:1003C00087165F1BE5295D180716DF18E929DD1878
:1003D0008715E6300E02031C012A5F1D05165F1DFE
:1003E00085165F1D0514DF1D85145F1E87145F1EB3
:1003F00007155F1E07145F1E87165F1F0716DF1C99
:1004000087158F08031908008F018501870155089A
:10041000DE00FF23D5005608DE00FF23D600570874
:10042000DE00551CFF23D7005808DE00D51CFF2333
:10043000D8005908DE00551DFF23D9005A08DE00F8
:10044000D51DFF23DA005B08DE00551EFF23DB000D
:100450005F1D442AC11B3F2AC11C0512C11C332A3F
:10046000051258190516CB0B552A5608CB00C101A9
:10047000D51BC114D81BC1105818C110552A05121C
:10048000CB0B552AC103552AC108031905160319B8
:10049000552ACB0B552AD51BC1035508CB00D518BF
:1004A0005C14D51E5C10D51D5C105F1D712AC21B2B
:1004B0006C2AC21C8512C21C602A85125818851627
:1004C000CC0B822A5608CC00C201D61BC2145A1883
:1004D000C210D619C210822A8512CC0B822AC203FE
:1004E000822AC208031985160319822ACC0B822A94
:1004F000D61BC2035608CC00D61ADC14561DDC10DD
:10050000561FDC105F1D9E2AC31B992AC31C0510B1
:10051000C31C8D2A05105A190514CD0BAF2A570894
:10052000CD00C301D71BC314D51AC310D719C310EC
:10053000AF2A0510CD0BAF2AC303AF2AC308031996
:1005400005140319AF2ACD0BAF2AD71BC3035708D5
:10055000CD00571A5C15571F5C11D71D5C11DF1DAC
:10056000CB2AC41BC62AC41C8510C41CBA2A8510F9
:10057000D51B8514CE0BE72A5808CE00C401D81B22
:10058000C414D71AC410D819C410E72A8510CE0B8A
:10059000E72AC403E72ADF1FD62ACE0BE72A58082A
:1005A000CE00D51BDC15DA1FDC11E72AC4080319BD
:1005B00085140319E72ACE0BE72AD81BC403580871
:1005C000CE00581ADC15D81FDC11D81DDC115F1EB7
:1005D000032BC51BFE2AC51C8710C51CF22A8710D9
:1005E000D51A8714CF0B142B5908CF00C501D91B7E
:1005F000C514561AC510D81BC510142B8710CF0B65
:10060000142BC503142BC508031987140319142BC5
:10061000CF0B142BD91BC5035908CF00D91B5C166F
:10062000D91F5C12D91C5C125F1E302BC61B2B2BF2
:10063000C61C0711C61C1F2B0711D71A0715D00B94
:10064000412B5A08D000C601DA1BC614D51AC610B1
:10065000D619C610412B0711D00B412BC603412BD5
:10066000C608031907150319412BD00B412BDA1BC0
:10067000C6035A08D0005A1ADC165A1EDC12DA1FBA
:10068000DC125F1E5D2BC71B582BC71C0710C71C35
:100690004C2B071059190714D10B6E2B5B08D10096
:1006A000C701DB1BC714D719C710DB19C7106E2B86
:1006B0000710D10B6E2BC7036E2BC7080319071445
:1006C00003196E2BD10B6E2BDB1BC7035B08D1000C
:1006D000DB195C17DB1D5C135B1E5C135F1E8A2B32
:1006E000C81B852BC81C8712C81C792B8712581968
:1006F0008716D20B9B2B5608D200C801D91BC814F1
:100700005A19C810551AC8109B2B8712D20B9B2B55
:10071000C8039B2BC8080319871603199B2BD20B00
:100720009B2BD71BC8035908D200561ADC17561E3C
:10073000DC13DA1FDC135F1FB72BC91BB22BC91CDC
:100740000712C91CA62B071255190716D30BD12B5C
:100750005808D300C901D61BC914D91AC910D81911
:10076000C910D12B0712D30BD12BC903D12B5F1C7E
:10077000C22BD30BD12B5708D300D61B5D14D81F27
:100780005D10D12BC908031907160319D12BD30B00
:10079000D12BD51AC9035808D300D61B5D14D81F16
:1007A0005D10DF1CED2BCA1BE82BCA1C8711CA1C6D
:1007B000DC2B8711D51B8715D40B08005508D400F6
:1007C000CA01D51BCA14561ACA10D619CA10080075
:1007D0008711D40B0800CA030800CA08031987153B
:1007E00003190800D40B0800D81BCA035608D4000C
:1007F000591ADD14591EDD10DA1FDD100800C00182
:10080000DE080319DE035E184014DE1A40144008A7
:10081000C0015E1C4014DE1E4014C005C00C5E0CFE
:020820000800CE
:084000000D00030007000000A1
:02400E00CC33B1
:10420000010078007A007C007E007B0079007F004E
:104210007D007A0078007E007C00FF00FF00FF0038
:104220000000F200F600FA00FE00F200F600FA00CC
:10423000FE00F200F600FA00FE00FF00FF00FF00A3
:10424000030005000500050005000900090009003C
:1042500009000D000D000D000D00FF00FF00FF0024
:10426000FF00FF00FF00FF00FF00FF00FF00FF0056
:10427000FF00FF00FF00FF00FF00FF00FF00FF0046
:10428000FF00FF00FF00FF00FF00FF00FF00FF0036
:10429000FF00FF00FF00FF00FF00FF00FF00FF0026
:1042A000FF00FF00FF00FF00FF00FF00FF00FF0016
:1042B000FF00FF00FF00FF00FF00FF00FF00FF0006
:1042C000FF00FF00FF00FF00FF00FF00FF00FF00F6
:1042D000FF00FF00FF00FF00FF00FF00FF00FF00E6
:1042E0000200BA00FF00FF00FF00FF00FF00FF0018
:1042F000FF00FF00FF00FF00FF00FF00FF00DD00E8
:00000001FF
